:020000040000fa
:080000000001040000000000f3
:020000040000fa
:100200002f80200080bf2000000188000000000037
:10021000050007000c000700b20202000000000009
:100220000040da000000fe004440a9000000200069
:100230000000e0000300320000002000a001880060
:100240004440a80000000600e02e2000010020002d
:100250001600370062004000e080480091018800ed
:100260009001ba0062004000e080480091018800df
:100270009002ba0062004000e08048000002eb00fb
:100280006028e10005003a008301e900070033001f
:10029000038009000059eb00040037006128e100e9
:1002a000010032000082eb00050007009101880088
:1002b0001001ba000200e000e6ff3a00000005006d
:1002c000910188008002780062004000e0804800d0
:1002d0003559ba008301e900080032002559ba00f7
:1002e0008301e900050032000400e000f4ff320061
:1002f00015d9ba008301e900f1ff3a0000000600b9
:10030000809fbe00821f78003400f80000c0b30058
:10031000a00188000000fa008460a90000c8bf00a6
:100320000004e000030032000040eb0000e8b700ea
:100330000200370010c0b30000e8b70000c8bf00db
:1003400061406000614060000040400000404000ab
:10035000004040000040400000414000112d2000be
:1003600091407800f0cdb30000c060000240700002
:10037000d1e2b7000080fa003400f9004f017800a4
:100380004f00be00004006000000fa00f000200010
:1003900030168800de82a900dea2a900cda2a90045
:1003a000d322a800e282a9000080fa000000060023
:1003b0000000fa0040012000570007008000eb0019
:1003c0000003200037000700500020005200070003
:1003d0008000eb00000320003200070050002000e6
:1003e0004d0007008000eb00000320002d000700f7
:1003f00050002000480007008000eb0000022000b1
:100400002800070050002000430007008000eb0098
:10041000e0022000100007008000eb0080002000b8
:100420000d0007008000eb00d00020000a0007004c
:100430008000eb0060002000070007008000eb0058
:1004400020002000040007005000200032000700b8
:100450000080fa00000006000200fa00004f780059
:10046000114798001e4090008000fb001e80fb009a
:100470000c0007001e4090008000fb001e80fb0067
:10048000000040000000400000004000000040006c
:1004900004000700200020001f0007000080fa0071
:1004a000000006000200fa00004f78001147980093
:1004b0001e80fb00501688001e40900061406000c6
:1004c00061406000004040000040400000404000ab
:1004d0000040400000414000212e20009140780063
:1004e000f0cdb30000c0600002407000e2e2b7004f
:1004f0000000eb0008000700e282a8000000eb000b
:1005000005000700e282a900100020000200070099
:100510000080fa00000006000400fa0010079800ae
:100520000b0037000000eb00000f780002003700de
:10053000000000001e0fe8000080eb009e0f10007e
:10054000fbff3a001e0090000000e9001007980031
:100550001e0090000000e000f2ff3a000080fa0068
:10056000000006000000fa0087ff070090ff070068
:1005700083e0a80042c0bf007f40600001c4b30018
:100580000140700042e0b7000000eb002008880046
:100590000000eb00000888000080eb0010088800d5
:1005a00000032800200888005109200091407800ad
:1005b000f0c8b30000c0600001c3b3000140700088
:1005c00095e0b7008460a9008c60a80011c0b3005a
:0c05d000f0c4b300a0ff0700ffff3700dd
:020000040000fa
:10000800f6020000f6020000f6020000f602000008
:10001800f6020000f6020000f6020000f6020000f8
:10002800f6020000f6020000f6020000f6020000e8
:10003800f6020000f6020000f6020000f6020000d8
:10004800f6020000f6020000f6020000f6020000c8
:10005800f6020000f6020000f6020000f6020000b8
:10006800f6020000f6020000f6020000f6020000a8
:10007800f6020000f6020000f6020000f602000098
:10008800f6020000f6020000f6020000f602000088
:10009800f6020000f6020000f6020000f602000078
:1000a800f6020000f6020000f6020000f602000068
:1000b800f6020000f6020000f6020000f602000058
:1000c800f6020000f6020000f6020000f602000048
:1000d800f6020000f6020000f6020000f602000038
:1000e800f6020000f6020000f6020000f602000028
:0800f800f6020000f602000010
:020000040000fa
:10010800f6020000f6020000f6020000f602000007
:10011800f6020000f6020000f6020000f6020000f7
:10012800f6020000f6020000f6020000800100005e
:10013800f6020000f6020000f6020000f6020000d7
:10014800f6020000f6020000f6020000f6020000c7
:10015800f6020000f6020000f6020000f6020000b7
:10016800f6020000f6020000f6020000f6020000a7
:10017800f6020000f6020000f6020000f602000097
:10018800f6020000f6020000f6020000f602000087
:10019800f6020000f6020000f6020000f602000077
:1001a800f6020000f6020000f6020000f602000067
:1001b800f6020000f6020000f6020000f602000057
:1001c800f6020000f6020000f6020000f602000047
:1001d800f6020000f6020000f6020000f602000037
:1001e800f6020000f6020000f6020000f602000027
:0801f800f6020000f60200000f
:020000040000fa
:1005dc000008000002000000000000000000000005
:020000040000fa
:0405ec000000fe000d
:00000001FF
